:020000040000FA
:0608000009EF11F01200E7
:02082A000000CC
:04082C0000018B91AB
:100830008B93200E8C6F080E916F8DC08FF08EC041
:1008400090F08F1F901F120000018BB10FD000019C
:10085000BCB10CD00001C36B0001010EC26F0001DE
:100860009A0EC16FE9EC0DF000018B8100018BB392
:100870000DD00001BCB194D10001C06B00019A0EF3
:10088000BF6FDDEC0DF000018B831200915102E08F
:1008900091071200080E916F8C5117E00001BCA95E
:1008A00077D100018C07BBC028F0296A28BE2968CF
:1008B0008D5128248D6F8E5129208E6F030E8D2728
:1008C000000E8E230001BC9963D1200E1F6E206A9A
:1008D0008DC01AF08EC01BF042EC10F01AC08DF0E3
:1008E0001BC08EF01AC028F01BC029F0200E1F6E0E
:1008F000206A42EC10F016C028F017C029F0173417
:1009000009E228501008000E295404E200018D2B42
:10091000000E8E2300018D518F1902E18E51901926
:1009200001E131D18DC08FF08EC090F0200E9D6F0F
:100930009C6F9B6F9A6F996F990EE66E000EE66E34
:100940008DC0E6FF8EC0E6FFCDEC0CF0E552E5521F
:10095000E552E5520001810E866F0C0E876F000E86
:10096000886F15EC08F00001050E986F0001980ED5
:10097000846F000E856FA4EC07F00001200E9D6FC0
:100980009C6F9B6F9A6F996F8DC028F08EC029F075
:10099000030ED89028362936E806FBE10A0E1F6EB2
:1009A000206A28C01AF029C01BF042EC10F01AC0CF
:1009B00028F01BC029F0200E2826000E29222850DE
:1009C00000018D25946F29508E21956F8DC028F0E0
:1009D0008EC029F0030ED89028362936E806FBE1B0
:1009E0000A0E1F6E206A28C01AF029C01BF042ECC4
:1009F00010F016C028F017C029F0173409E228506B
:100A00000508000E295404E20001942B000E9523E2
:100A1000990EE66E000EE66E94C0E6FF95C0E6FF06
:100A2000CDEC0CF0E552E552E552E5520001890E9D
:100A3000866F0C0E876F000E886F15EC08F00001B2
:100A4000050E986F0001980E846F000E856FA4EC60
:100A500007F00001200E9D6F9C6F9B6F9A6F996F3E
:100A6000110E8D25926F010E8E21936F990EE66EF9
:100A7000000EE66E92C0E6FF93C0E6FFCDEC0CF0F0
:100A8000E552E552E552E5520001910E866F0C0EDB
:100A9000876F000E886F15EC08F00001050E986F47
:100AA0000001980E846F000E856FA4EC07F0000122
:100AB000200E9D6F9C6F9B6F9A6F996F8DC028F071
:100AC0008EC029F0030ED89028362936E806FBE1BF
:100AD0000A0E1F6E206A28C01AF029C01BF042ECD3
:100AE00010F01AC028F01BC029F0EC0E2826010EC9
:100AF0002922285000018D25966F29508E21976F4D
:100B00008DC028F08EC029F0030ED89028362936E3
:100B1000E806FBE10A0E1F6E206A28C01AF029C001
:100B20001BF042EC10F016C028F017C029F0173463
:100B300009E228500508000E295404E20001962B12
:100B4000000E9723990EE66E000EE66E96C0E6FF45
:100B500097C0E6FFCDEC0CF0E552E552E552E552C8
:100B60000001990E866F0C0E876F000E886F15ECD2
:100B700008F00001050E986F0001980E846F000EBA
:100B8000856FA4EC07F00001200E8C6F8D6B8E6BCF
:100B90000001BCB105D000019A0EC46FF7EC0DF056
:020BA000120041
:0E0BA200031B5B66031B5B4A020D0A5750499A
:100BB0004344454D20485043204578706C6F726522
:100BC000720A0D004D6963726F6368697020546525
:100BD00063686E6F6C6F677920496E632E0A0D0033
:100BE00044656D6F206669726D776172652076313C
:100BF0002E30310A0D00417072696C2031342C2086
:100C0000323030350A0D000B526F737320466F730C
:100C10006C65720A0D00691B5B363B316654656D6D
:100C20007065726174757265202843656C736975AF
:100C300073293A0A0D0054656D706572617475729E
:100C400065202846616872656E68656974293A0A8C
:100C50000D0054656D706572617475726520284B66
:100C6000656C76696E293A0A0D0054656D7065727F
:100C70006174757265202852616E6B696E65293AE0
:100C800000071B5B363B323766071B5B373B32374F
:100C900066071B5B383B323766071B5B393B3237D5
:100CA00066211B5B31313B3166504F5420566F6CCF
:100CB000746167653A200A0D00504F542056616CEC
:100CC00075653A00081B5B31313B313466081B5BAC
:100CD00031323B313466591B5B31343B31665072E3
:100CE000657373206B6579202731272074686F75D1
:100CF0006768202738270A0D004C4544733A2020A6
:100D00002044312020204432202020443320202041
:100D10004434202020443520202044362020204404
:100D20003720202044380A0D005374617475733ADB
:100D30002000071B5B31363B3966054F6E202020B3
:100D400000054F6666202000131B5B31383B31667F
:100D5000427574746F6E205242303A2000081B5B5B
:100D600031383B3133660B507265737365642020F4
:100D70002020000B4E6F74207072657373656400E1
:100D8000241B5B32323B31665072657373202762DD
:100D90002720746F20656E74657220626F6F7420F7
:100DA0006D6F64652E00121B5B32303B31665469F7
:100DB0006D653A200007081B5B32303B3131663FDE
:100DC0001B5B373B3166456E746572696E672062E6
:100DD0006F6F74206D6F64652077696C6C20666F2F
:100DE000726365207468652064656D6F2066697242
:100DF0006D7761726520746F2073746F700A0D00D7
:100E00005366756E6374696F6E696E672E20416EEE
:100E1000792070726F6772616D6D696E67206F7097
:100E200065726174696F6E207468657265206166B1
:100E3000746572206D61790A0D0064657374726F58
:100E400079207468652064656D6F20636F64652E1A
:100E50000A0D0A0D001F446F20796F752077616EAF
:100E60007420746F20656E74657220626F6F7420D9
:060E70006D6F64653F0098
:0A0E760083C082F0000E0001796FC6
:100E80007A6B776F786B8193AB6A900EAB6EAC6ABE
:100E9000240EAC6E83C0AFFF010C12000001815123
:100EA000020B43E0AC50020B40E07DC0E9FF7EC086
:100EB000EAFFEF50AD6E7F077F5134E1795177192A
:100EC00011E17A5178190EE177C007F078C008F087
:100ED000B5EC0BF0000E0001796F7A6B776F786BD1
:100EE000819323D077C0E9FF78C0EAFFEE52EECFBE
:100EF0007BF0EDCF7CF0030E7B257D6F000E7C2117
:100F00007E6F77C0E9FF78C0EAFFEFCF7FF077C050
:100F100007F078C008F0B5EC0BF07BC077F07CC030
:100F200078F003D07D2B000E7E23AB50040B03E141
:100F3000AB50020B08E0AB6A900EAB6EAC6A240EAD
:100F4000AC6E82C0AFFF120084C0E9FF85C0EAFF2B
:100F5000EF50286E296A010E2826000E2922020E63
:100F600028240001006F52EC0BF0F3CF7BF0F4CF9C
:100F70007CF00001F350F41057E07751781119E13B
:100F80007BC079F07CC07AF07BC077F07CC078F0D1
:100F900084C0E9FF85C0EAFFEFCF7FF0010E77251F
:100FA0007D6F000E78217E6F020E7D27000E7E235E
:100FB0001AD079C0E9FF7AC0EAFFEE527BC0EEFF9B
:100FC0007CC0EDFF84C0E9FF85C0EAFFEF50E66E0C
:100FD00079C0E9FF7AC0EAFFE552E750EF6E7BC0C7
:100FE00079F07CC07AF084C0E9FF85C0EAFFEF5059
:100FF0000001B06FB16B030E00017B250001AE6FE5
:10100000000E00017C210001AF6F010E000184255C
:101010000001AC6F000E000185210001AD6F99EC5D
:1010200008F000018183010C000C86C0F6FF87C028
:10103000F7FF88C0F8FF0800F550286E296A010EF6
:101040002826000E2922020E28240001006F52ECEF
:101050000BF0F3CF7BF0F4CF7CF00001F350F410F1
:1010600061E0775178111CE17BC079F07CC07AF0A7
:101070007BC077F07CC078F086C0F6FF87C0F7FFB2
:1010800088C0F8FF0800F5CF7FF0010E77257D6F4F
:10109000000E78217E6F020E7D27000E7E231DD06C
:1010A00079C0E9FF7AC0EAFFEE527BC0EEFF7CC058
:1010B000EDFF86C0F6FF87C0F7FF88C0F8FF080085
:1010C000F550E66E79C0E9FF7AC0EAFFE552E750D5
:1010D000EF6E7BC079F07CC07AF086C0F6FF87C0E7
:1010E000F7FF88C0F8FF0800F5500001B76FB86B34
:1010F000030E00017B250001B56F000E00017C216D
:101100000001B66F86C0B2F087C0B3F088C0B4F0FB
:101110000001B22B000EB323B42368EC09F00001E8
:101120008183010C000C12009EAA02D0AE50120066
:02113000000CB1
:0E1132000001B051B11101E1C9D0040EB05D51
:10114000000EB15911E2ACC0E9FFADC0EAFFEF50AB
:10115000AEC0E9FFAFC0EAFFEF6EAE2B000EAF23CB
:10116000AC2BAD23B007B1D0080EB05D000EB15965
:1011700022E2ACC0E9FFADC0EAFFEECF28F0EECF2F
:1011800029F0EECF2AF0EFCF2BF0AEC0E9FFAFC0D1
:10119000EAFF28C0EEFF29C0EEFF2AC0EEFF2BC0F9
:1011A000EEFF040EAE27000EAF23040EAC27000E98
:1011B000AD23040E88D0100EB05D000EB15932E29E
:1011C000ACC0E9FFADC0EAFFEECF28F0EECF29F0CA
:1011D000EECF2AF0EECF2BF0EECF2CF0EECF2DF0AD
:1011E000EECF2EF0EFCF2FF0AEC0E9FFAFC0EAFF99
:1011F00028C0EEFF29C0EEFF2AC0EEFF2BC0EEFF95
:101200002CC0EEFF2DC0EEFF2EC0EEFF2FC0EEFF74
:10121000080EAE27000EAF23080EAC27000EAD233C
:10122000080E51D0ACC0E9FFADC0EAFFEECF28F008
:10123000EECF29F0EECF2AF0EECF2BF0EECF2CF050
:10124000EECF2DF0EECF2EF0EECF2FF0EECF30F030
:10125000EECF31F0EECF32F0EECF33F0EECF34F010
:10126000EECF35F0EECF36F0EFCF37F0AEC0E9FF7E
:10127000AFC0EAFF28C0EEFF29C0EEFF2AC0EEFF94
:101280002BC0EEFF2CC0EEFF2DC0EEFF2EC0EEFFF8
:101290002FC0EEFF30C0EEFF31C0EEFF32C0EEFFD8
:1012A00033C0EEFF34C0EEFF35C0EEFF36C0EEFFB8
:1012B00037C0EEFF100EAE27000EAF23100EAC2786
:1012C000000EAD23100EB05F000EB15B32D71200DE
:1012D0000001B751B81101E188D0040EB75D000ECE
:1012E000B85915E2B2C0F6FFB3C0F7FFB4C0F8FFBB
:1012F0000800F550B5C0E9FFB6C0EAFFEF6EB52BA8
:10130000000EB623B22BB323B423B7076CD0080E5C
:10131000B75D000EB85929E2B2C0F6FFB3C0F7FFBF
:10132000B4C0F8FF0900F5CF28F00900F5CF29F087
:101330000900F5CF2AF00800F5CF2BF0B5C0E9FF82
:10134000B6C0EAFF28C0EEFF29C0EEFF2AC0EEFFBC
:101350002BC0EEFF040EB527000EB623040EB227F5
:10136000000EB323B423040E3CD0B2C0F6FFB3C0CA
:10137000F7FFB4C0F8FF0900F5CF28F00900F5CF5A
:1013800029F00900F5CF2AF00900F5CF2BF009006C
:10139000F5CF2CF00900F5CF2DF00900F5CF2EF098
:1013A0000800F5CF2FF0B5C0E9FFB6C0EAFF28C0AE
:1013B000EEFF29C0EEFF2AC0EEFF2BC0EEFF2CC0CF
:1013C000EEFF2DC0EEFF2EC0EEFF2FC0EEFF080E89
:1013D000B527000EB623080EB227000EB323B423A0
:0C13E000080EB75F000EB85B73D7120058
:0413EC00010EC26EBE
:1013F000C16A830EC06E0001400E606F61C063F071
:1014000062C064F0631F641F12009EAC49D19E9CB1
:101410000001605108E060076151C324616F6251AF
:10142000C420626F120061C028F062C029F0060E6D
:10143000D89029322832E804FBE128C061F029C0A5
:1014400062F000012850631902E16251641901E160
:1014500021D161C063F062C064F00001CD0E866FDF
:101460000C0E876F000E886F15EC08F00001200E3F
:10147000766F756F746F736F726F720EE66E000E1B
:10148000E66E61C0E6FF62C0E6FFCDEC0CF0E5520F
:10149000E552E552E5520001050E716F0001710E33
:1014A000846F000E856FA4EC07F00001C40E866FF8
:1014B0000C0E876F000E886F15EC08F00001200EEF
:1014C000766F756F746F726F050E1A6E1B6A61C04E
:1014D0001FF062C020F068EC10F018C065F019C071
:1014E00066F01F68030E206E18C01AF019C01BF0BA
:1014F000E2EC10F01AC065F01BC066F00001676BEB
:10150000686B720EE66E000EE66E1AC0E6FF1BC038
:10151000E6FFCDEC0CF0E552E552E552E552000154
:101520002E0E736F050E1A6E1B6A61C01FF062C02B
:1015300020F068EC10F018C065F019C066F01F6864
:10154000030E206E18C01AF019C01BF0E2EC10F068
:1015500016C065F017C066F000010A0E6603F3CFEF
:1015600066F06503F3CF65F0F4506627676B686B30
:10157000F3CF69F066C06AF067C06BF068C06CF0CA
:101580001D68030E1E6E1F6A206AF3CF18F066C036
:1015900019F067C01AF068C01BF0BEEC10F018C05C
:1015A00069F019C06AF01AC06BF01BC06CF0740EC1
:1015B000E66E000EE66E18C0E6FF19C0E6FFCDEC41
:1015C0000CF0E552E552E552E55265C069F066C09F
:1015D0006AF067C06BF068C06CF01D68030E1E6E89
:1015E0001F6A206A65C018F066C019F067C01AF05B
:1015F00068C01BF0BEEC10F014C069F015C06AF0B2
:1016000016C06BF017C06CF00A0E1D6E1E6A1F6AC2
:10161000206A14C018F015C019F016C01AF017C0CF
:101620001BF086EC10F014C069F015C06AF016C00B
:101630006BF017C06CF01D68030E1E6E1F6A206AE7
:1016400014C018F015C019F016C01AF017C01BF01E
:10165000BEEC10F018C069F019C06AF01AC06BF047
:101660001BC06CF0750EE66E000EE66E18C0E6FF4D
:1016700019C0E6FFCDEC0CF0E552E552E552E5521B
:101680000001050E716F0001710E846F000E856FF1
:10169000A4EC07F00001400E606F616B626B1200FA
:0416A000C2821200F0
:0C16A40000507E0810E3000E016E0A0EDC
:1016B000026E01C0E9FF02C0EAFFEF50056EE8507C
:1016C0007F0BFF0F066E055003E1F36AF46A120008
:1016D00005BE42D00650D880005408E201C00DF08B
:1016E00002C00EF074D80009E4E136D00650005C68
:1016F0000EE101C0E9FF02C0EAFFEF8E010E0124F6
:10170000286E000E022028C0F3FFF46E1200810E36
:101710000024E66E01C0E9FF02C0EAFFE552E7508F
:10172000EF6E010E0124036E000E0220046E0028ED
:10173000296AE8500126295002220050065CE66E14
:1017400001C0E9FF02C0EAFFE552E750EF6E03C0B7
:10175000F3FF04C0F4FF120005507F0B286E296AC6
:10176000E850012629500222A4D707C0E9FF08C08B
:10177000EAFFE906000EEA5AEF9E1200000E096E1B
:101780000A0E0A6E0B68020E0C6E7F0ED8800B5488
:10179000000E0C540EE209C0E9FF0AC0EAFF7F0EFA
:1017A000EF6E0926000E0A227F0E0B5E000E0C5A09
:1017B000ECD709C0E9FF0AC0EAFF0BC0EFFF0950F0
:1017C0000B24E96E0A500C20EA6EEF6A12000DC07D
:1017D000E9FF0EC0EAFFEF500D240F6E000E0E2041
:1017E000106EEF50116E0FC0E9FF10C0EAFFEF500E
:1017F000126EE85001E1000C1150800B03E1125011
:10180000800B01E0000C11507F0B7F0801E1000C00
:1018100011501224136EE8507F081BE20DC0E9FF3F
:101820000EC0EAFF7F0EEF6E0D26000E0E22125044
:10183000296A12500F26295010220D500F5C286E75
:101840000E5010580DC0E9FF0EC0EAFF28C0EFFF90
:101850007F0C0DC0E9FF0EC0EAFF13C0EFFFEF5091
:02186000120074
:0E1862008C68956A12000001320E866F0D0E22
:10187000876F000E886F15EC08F08CA007D0000170
:101880003A0E866F0D0E876F000E06D00001410ED6
:10189000866F0D0E876F000E886F15EC08F08CA216
:1018A00007D000013A0E866F0D0E876F000E06D02E
:1018B0000001410E866F0D0E876F000E886F15ECCC
:1018C00008F08CA407D000013A0E866F0D0E876FCA
:1018D000000E06D00001410E866F0D0E876F000EC0
:1018E000886F15EC08F08CA607D000013A0E866FC1
:1018F0000D0E876F000E06D00001410E866F0D0E93
:10190000876F000E886F15EC08F08CA807D00001D7
:101910003A0E866F0D0E876F000E06D00001410E45
:10192000866F0D0E876F000E886F15EC08F08CAA7D
:1019300007D000013A0E866F0D0E876F000E06D09D
:101940000001410E866F0D0E876F000E886F15EC3B
:1019500008F08CAC07D000013A0E866F0D0E876F31
:10196000000E06D00001410E866F0D0E876F000E2F
:10197000886F15EC08F08CAE07D000013A0E866F28
:101980000D0E876F000E06D00001410E866F0D0E02
:0A199000876F000E886F15EF08F056
:06199A00D9CFE6FFDACF11
:1019A000E6FFFA0EE3CFD9FFFB0EE3CFDAFFFD0E21
:1019B000E35209E72D0EDE6EFC0EE31EE32AFD0E58
:1019C000D8B4E306E31EE652E652E652FD0EE124E9
:1019D000E76EFF0EE220E46EE652F70EE3CFE6FF7D
:1019E000F70EE3CFE6FF3DEC0DF0F90EE124E96ED2
:1019F000FF0EE220EA6E2DEC0DF00AE12AEC0DF06C
:101A000009E12DEC0DF008E12AEC0DF007E108D01A
:101A100038EC0DF033EC0DF038EC0DF033EC0DF04C
:101A200038EC0DF0DE6AF90EE126FF0EE222FF0E21
:101A3000E3CFDAFFE552FF0EE3CFD9FFE552FC0E0C
:101A4000E124E96EFF0EE220EA6EEECFF3FFEFCF66
:101A5000F4FF1200EF380F0B1200EF500F0B02E1F2
:101A6000EE52D8841200EF380F0B300FDE6E1200EA
:101A7000EE500F0B300FDE6E1200FC0EE3CFE9FFCD
:101A8000FD0EE3CFEAFF100EE66EEE6AEE6AEF6A35
:101A9000D890FD0EE336FE0EE336ED36ED36EF362A
:101AA000FF0EE30609E05EEC0DF0EE525EEC0DF089
:101AB000EE525EEC0DF0EDD7E56E1200030EEF2452
:0E1AC000E8B6EF6E300EEF24E8BEEF6E000CBD
:021ACE00000115
:101AD000BC6BBD6B8B868B8894869488C78E280ED2
:101AE000C66EC78CBEC0C8FF9E9612009EA664D06C
:101AF0009E960001BCA310D0BCB95ED0BDA139D068
:101B0000BDA33CD0BDB503D0C5AC12D015D0BDBB74
:101B100027D0C5AC4AD019D0BCA525D0BCB94CD073
:101B2000BDA127D0BDA32AD0BDB508D0C5BC04D067
:101B3000BAC0C9FFBD851200BD932CD0BDB708D077
:101B4000C5BC03D0BBC0C9FF22D0BD93BD9522D078
:101B5000BDBB06D0C5AC29D0BD93BD95BD971AD0ED
:101B6000BC89BC911200BCA727D0BCB925D0BDB19F
:101B700003D0C580BD811200BDB304D0B9C0C9FF78
:101B8000BD831200BDB708D0C5BC03D0C586BD87D4
:101B90001200BD93C5821200BDB905D0C596C58A95
:101BA000C588BD891200BDBB03D0C584BD8B1200A2
:101BB000C9CFBBF0BC89BC911200FE0E0001BF155D
:101BC000B96FC0C0BAF0BD6BBC6BBC81BC839E86D4
:101BD0001200FE0E0001C115B96FC2C0BAF0C3C039
:101BE000BBF0BD6BBC6BBC81BC859E861200010E38
:101BF0000001C411B96FBD6BBC6BBC81BC879E86F4
:021C00001200D0
:0E1C02000F0ECD6E800ECF6ECE6A0001A16B6C
:101C1000A1C0A0F0A1C09EF012009EA065D09E9031
:101C2000CF8E00019E2B00019E513B0812E2000165
:101C30009E6B0001A02B0001A0513B080AE20001AD
:101C4000A06B0001A12B0001A151170802E20001C5
:101C5000A16B00019E5100019F5D46E09EC09FF078
:101C60000001B60E866F0D0E876F000E886F15ECA3
:101C700008F0A30EE66E000EE66E0001A051E66EBF
:101C8000E66ACDEC0CF0E552E552E552E552000172
:101C9000A45105E1A3C0A4F00001300EA36F000120
:101CA0003A0EA56FA60EE66E000EE66E00019E517E
:101CB000E66EE66ACDEC0CF0E552E552E552E552EF
:101CC0000001A75105E1A6C0A7F00001300EA66FE4
:101CD0000001A86B0001050EA26F0001A20E846F27
:0A1CE000000E856FA4EC07F012005F
:061CEA0081B003D0FC6A8A
:101CF00002EF00F0BEEC0BF0F8EC10F000012B0E40
:101D0000836F3BEC07F04AEC0FF031EC0CF034EC55
:101D10000CF0F6EC09F0F3EC0FF000017F0EBE6F53
:101D200067EC0DF016EC04F001EC0EF04EEC07F051
:101D300076EC0DF0FFEC10F0000908E005EC0AF07D
:101D40000DEC0EF013EC10F024EC04F094EC08F021
:101D50000001CF6F0001CF51620A31E05A0A2BE037
:101D60000F0A25E0010A1FE0030A19E0010A13E047
:101D7000070A0DE0010A07E0030A01E023D08C7096
:101D800034EC0CF01FD08C7234EC0CF01BD08C7443
:101D900034EC0CF017D08C7634EC0CF013D08C783B
:101DA00034EC0CF00FD08C7A34EC0CF00BD08C7C33
:101DB00034EC0CF007D08C7E34EC0CF003D0E4EC67
:081DC0000EF000D0B3D71200B1
:081DC8000001A20E866F0B0E54
:101DD000876F000E886F15EC08F00001A60E866F65
:101DE0000B0E876F000E886F15EC08F00001A20E35
:101DF000866F0B0E876F000E886F15EC08F00001E0
:101E0000AD0E866F0B0E876F000E886F15EC08F015
:101E10000001BF0E866F0D0E876F000E886F15ECE8
:101E200008F00001000E866F0E0E876F000E886F9F
:101E300015EC08F00001550E866F0E0E876F000E30
:101E4000886F15EC08F04EEC07F076EC0DF094EC92
:101E500008F00001D26F0001D25109E0790A03E0D5
:101E6000200A01E005D0FC6A02EF00F011D010D08A
:101E70004AEC0FF0F6EC09F005EC0AF0F3EC0FF089
:101E800034EC0CF016EC04F024EC04F002D000D09A
:041E9000DAD712008B
:0C1E94000001A20E866F0B0E876F000E7F
:101EA000886F15EC08F00001A60E866F0B0E876F89
:101EB000000E886F15EC08F00001A20E866F0B0E65
:101EC000876F000E886F15EC08F00001AD0E866F6D
:101ED0000B0E876F000E886F15EC08F00001160ED0
:101EE000866F0C0E876F000E886F15EC08F00001EE
:101EF000A10E866F0C0E876F000E886F15EC08F030
:101F00000001D60E866F0C0E876F000E886F15ECE1
:101F100008F00001480E866F0D0E876F000E886F67
:101F200015EC08F00001800E866F0D0E876F000E15
:101F3000886F15EC08F00001A60E866F0D0E876FF6
:081F4000000E886F15EF08F098
:081F48002A0EF66E080EF76E7A
:101F5000000EF86E00010900F550CA6F0900F55037
:101F6000CB6F03E1CA6701D03DD00900F550C56FC2
:101F70000900F550C66F0900F550C76F0900090048
:101F8000F550E96E0900F550EA6E090009000900F4
:101F9000F550C86F0900F550C96F09000900F6CF68
:101FA000CCF0F7CFCDF0F8CFCEF0C5C0F6FFC6C06D
:101FB000F7FFC7C0F8FF0001C85302E1C95307E0AB
:101FC0000900F550EE6EC807F8E2C907F9D7CCC092
:101FD000F6FFCDC0F7FFCEC0F8FF0001CA07000E24
:061FE000CB5BBFD712002D
:0A1FE60000015D0E866F0D0E876F7F
:101FF000000E886F15EC08F081A007D00001730E69
:10200000866F0D0E876F000E06D00001660E866F7C
:102010000D0E876F000E886F15EC08F08150010BD4
:102020000001D16F120081A013D00001D15125E130
:1020300000015D0E866F0D0E876F000E886F15EC28
:1020400008F00001730E866F0D0E876F000E12D020
:102050000001D15112E000015D0E866F0D0E876FF9
:10206000000E886F15EC08F00001660E866F0D0EED
:10207000876F000E886F15EC08F08150010B00018E
:04208000D16F12000A
:0C208400226A20AE4BEF10F01F6C201EF3
:10209000E86A2022221E1BAE53EF10F01A6C1B1EA2
:1020A000E86A1B22221EE2EC10F01BBE63EF10F068
:1020B00022AE000C1A6C1B1EE86A1B22166C171E3F
:1020C000E86A1722000C22BE5AEF10F02388FF0C9A
:1020D0001AC026F01A501F02F4CF19F0F3CF18F0EF
:1020E0001B502002F4CF1BF0F3CF1AF01F02F35065
:1020F0001926F4501A22E86A1B2226502002F350B7
:0C2100001926F4501A22E86A1B22000C79
:04210C0018501D0248
:10211000F3CF14F0F4CF15F01E02F3501526000E85
:10212000F420166E18501F02F3501626000EF420ED
:10213000176E18502002F350172619501D02F35045
:102140001526F4501622000E172219501E02F350C5
:102150001626F450172219501F02F35017261A5052
:102160001D02F3501626F45017221A501E02F35087
:0C21700017261B501D02F350172612000A
:04217C00176A166A5E
:10218000156A146A200EE76ED890183619361A367A
:102190001B3614361536163617361D50145C1E5075
:1021A00015581F5016582050175809E31D50145E3B
:1021B0001E50155A1F50165A2050175A182AE72E2B
:0421C000E4D712004E
:0C21C400176A166A100EE76ED8901A36E3
:1021D0001B36163617361F50165C2050175805E36D
:1021E0001F50165E2050175A1A2AE72EF0D71200F9
:1021F000470ED56EC70ED66ED58EF2941200F2A49D
:1022000007D00001C80ED06FE850D626F294010C1A
:02221000000CC0
:0E2212001DEE00F02DEE00F0F86A239CA4EC07
:0A2220000FF075EC0EF0FDD7120070
:020000040030CA
:0C000000FFF6EEFEFFFF8BFFFF80FFA06D
:00000001FF
